:020000020000FC
:1000000012C0189518951895189518954AC04BC0A8
:1000100018951895189549C018951895189518951C
:100020001895189518950FE50DBF04E00EBF0FEF5A
:1000300004BBA0E680E29EE49BBD8ABD8CED95E00A
:1000400099BD88BD09B7086109BF0AE00EBD03E389
:1000500009B900E000BD06E800BD579A549A7894AB
:100060001A32F1F71127EE27FF27AA950E910053B8
:10007000E02F0E9100532AE0029FE00D0E910053F5
:1000800024E6029FE00DF11D88EE93E00E910053EF
:1000900021F0E80FF91F0A95FBCFF9BDE8BDA0E6F6
:1000A000DFCFA99A1895A99818950F930CB10D93C5
:0A00B0000A3209F4102F0F91189581
:00000001FF
